:020000040800F2
:10500000201A0020D550000849820008717A000853
:105010000000000000000000000000000000000090
:10502000000000000000000000000000B18E000839
:1050300000000000000000008D870008CD8F0008F0
:10504000E7500008E7500008E7500008E750000864
:10505000E7500008295B0008E7500008E750000807
:1050600000000000E7500008515A0008E75000080F
:10507000E7500008C57E000800000000E750000867
:1050800000000000E75000080000000000000000E1
:10509000E750000800000000E7500008E750000853
:1050A000E7500008E7500008E75000086197000843
:1050B000E7500008E7500008000000000000000072
:1050C0000348854600F060FC004800478DA50008B5
:1050D000201A00200448804704480047FEE7FEE706
:1050E000FEE7FEE7FEE7FEE769900008C150000812
:1050F00030B50B46014600202022012409E00D4670
:10510000D5409D4205D31D469540491B25469540F7
:1051100040191546521E002DF1DC30BDF0B51FB40C
:105120000646002082B005464024019100901BE015
:10513000019922460F46304600F04EFB049A059B2B
:10514000801A994110D310461946224600F034FBCC
:10515000361A8F410197224601200021009F00F05E
:105160002BFB38184D4100902046641E0028DFDCE0
:10517000019B00982946324607B0F0BD03460B4319
:105180009B0703D009E008C9121F08C0042AFAD2FD
:1051900003E00B780370401C491C521EF9D2704783
:1051A000D2B201E00270401C491EFBD270470022BF
:1051B000F6E710B513460A4604461946FFF7F0FF16
:1051C000204610BD30B504460020034600E05B1CBD
:1051D000934203D2E05CCD5C401BF8D030BDF8B503
:1051E00002464A40D40F42004B0052085B089A42E4
:1051F00002D20246084611464A0023D0C30D4A0097
:10520000DDB2120EAD1A202D35DA49020126490A07
:10521000F6058A19002C00D0524220214F1B11465E
:10522000B9402A411018C20D9A4221D0002C17D043
:10523000012D08DCDA05801AD20F8019D207DBB203
:1052400000F0F6FAF8BDDA05801A012340001B06CB
:10525000C01880185A428018CA0F1043490007E04E
:105260004908C2071143DA05801A801940088018DE
:1052700000F0D6FAF8BD61000122511A001BF7E7D1
:105280000122D2075140AAE70122D2075040A6E7E7
:1052900070B502464A40D50F40004A00ED0740086D
:1052A0005208002814D0002A12D0C40DD30D410298
:1052B0000120C0055202490A520AE41A09181218BC
:1052C0007D34914201D3641C00E04900002C01DAD6
:1052D000002070BD0023914201D3891A0343400886
:1052E00049000028F7D100290AD0914202D10121BA
:1052F000C90705E0914201D2012101E00121C94322
:10530000E005C018401900F08BFA70BDF0B50746F3
:105310000846584087B0C00F049048000E46590018
:1053200040084908BC1A884105D2384631461E4615
:1053300017460B4602465800400810434CD0300D2B
:10534000039040055900400D490D0590401A029008
:10535000402872DA18030121000B09050843019067
:1053600004980092002805D00199524200208841FB
:1053700000920190029840210A1A0199009800F0C9
:105380001BFA05460C466B4607CB00F036FAC019EF
:105390007141039A0E0D0023D71756401A467A40E2
:1053A000164344D0049A002A2DD0029A012A039A67
:1053B00015DC1205C01A914101263605001C714109
:1053C000D20F059ED2070093019202962A462346E9
:1053D00000F074FA07B0F0BD38463146FAE716051A
:1053E000224A0F46B218C01AB74101210905001C14
:1053F0004F4100187F41114618187941E20F1043C0
:105400006D19644113E0E2076D0815436408C20793
:105410001443039A01261205C01A91413605001C57
:105420007141CE07400830434908C01851412A460F
:10543000234600F036FACDE7FFE70498012240004A
:10544000C117121A00238B4104983146C417381A29
:10545000A141EEE730B40124E407634030BC55E7D6
:1054600030B40124E407614030BC4FE70000E0FFA6
:10547000F0B51FB488B00B990998002448400999E9
:10548000C00F490049080991C0070B9900904900D5
:1054900049080B9109990898A64608431CD00B9916
:1054A0000A98084318D0099801244000420D48008A
:1054B000410D099824050003000B204309900B9827
:1054C0000003000B20430B9050181C494018002289
:1054D00001901446104605E0002001460DB0F0BDD5
:1054E000032801DA034600E003239C46C11A0AAEF2
:1054F0000AE05F0008ADED5B4F00F75B7D430027DE
:10550000AA187C41491C5B1E6145F2DD410004ABD9
:105510005A522104120C0A43240C401C0828DFDBD9
:10552000019802900099704601910090059B049AA1
:105530000799069800F0C2F9D0E700000DFCFFFFC4
:10554000F0B50C465C4085B0E40FE40703944C00D2
:1055500000266408590094464908024602962243F0
:1055600021D062460A431ED06200570D4A000E0346
:105570002303550D012402462C492405781B1B0BDF
:10558000360B401823432643614600901C46501AB0
:10559000B44103D30098401C009002E09218009898
:1055A0005B41002803DA0020014605B0F0BD002071
:1055B000012109050746864611E064461D46141B75
:1055C000B54106D36546521BB341744607430C43AD
:1055D000A646CD0740084908284392185B41054676
:1055E0000D43EAD11046184313D060461946504087
:1055F0007140084306D06046101AB34106D201221A
:10560000002306E000220123DB0702E00122D2434F
:105610005310009874460105381C6141029C039D9B
:105620000019694100F03DF9BFE70000FD030000EB
:10563000C217C10F504010B54018CA079623002169
:1056400000F0F6F810BD10B500229623114600F0C8
:10565000EFF810BD0EB5C217C10F5040CA07401871
:105660000021054B0293019200910A460B4600F07F
:1056700025F903B000BD0000330400000EB5054954
:105680000291002100910A460B46019100F016F9A3
:1056900003B000BD33040000410040020122400A73
:1056A000D205090E80187F2901DA0020704796295B
:1056B00003DC9622511AC8407047963988407047DB
:1056C00070B5CD0F4A0009030123090B1B051943CF
:1056D0000B4BED070024520D9A4201DA002070BDF9
:1056E000074B34339A4203DC9A1A00F075F802E053
:1056F0000449511888402C43F1D0404270BD00004D
:10570000FF030000CDFBFFFF4A0009030123090B43
:105710001B051943094B10B5520D9A4201DA0020BE
:1057200010BD064B34339A4203DC9A1A00F054F849
:1057300010BD03495118884010BD0000FF03000050
:10574000CDFBFFFFC20FD207400040080BD0C10DB8
:105750000723DB01C91840020905400A1143C208AA
:10576000400711437047002001467047CB0FDB070D
:10577000490010B5490802460A4307D00A0D07241C
:105780000903E401090B121B002A01DC002010BDF3
:10579000C900440F0C43C100E018D205801800F086
:1057A0003FF810BD0122D207002800DB101A0029A3
:1057B00000DB511A8142704710B5202A04DB0146F4
:1057C000203A9140002010BD914020239C1A0346AE
:1057D000E3401943904010BD10B5202A04DB084671
:1057E000203AD040002110BD0B46D340D0402024A9
:1057F000A21A91400843194610BD10B5202A06DBB5
:10580000CB170846203A1041C1170B4306E00B4660
:105810001341D0402024A21A91400843194610BDDC
:10582000002904DA401C490001D1400840007047BB
:1058300070B40024050C05D11024000402D1002905
:1058400021D01124050E01D100020834050F01D129
:105850000001241D850F01D18000A41C002801DB5C
:105860004000641C002908D020252E1B0D46F54061
:10587000A14000D001212943084301061B1B000A57
:10588000DB1D02D5002070BC7047DB05181880189E
:105890000029F8DA401C4900F5D170BC40084000EE
:1058A000704710B5002B08DA0024401C61419218A3
:1058B0005B411A4301D14008400010BDF0B51FB450
:1058C00082B005460C0003D0084604F009F802E057
:1058D00004F006F820300246009021462846FFF7E3
:1058E0006BFF049B059A04460F4618431143084377
:1058F00014D0184610431BD0009840210A1A1846AD
:105900000599FFF769FF05460E46009A0599049828
:10591000FFF752FF084305D0012004E02046394636
:1059200007B0F0BD0020C11705430E432C43374399
:1059300000990E986305401A7905E40A00220C4389
:10594000FD0A0A3002D500200146E9E701051019D9
:1059500069410C9C0D9D00196941FFF7A2FFDFE72B
:1059600010B5002904DB0124E40740428C412146A4
:10597000002B04DB1C460123DB075242A341994262
:1059800000D1904210BD0000064C0125064E05E0F6
:10599000E36807CC2B430C3C98471034B442F7D350
:1059A000FFF792FBFCA800081CA9000838B50446C4
:1059B000064805490068FFF79BFB604300E0401E76
:1059C00000900028FBD138BD40420F001C01002090
:1059D000F8B50446006881688907890F012902D15A
:1059E0000168C90722D18168114A1026114001259A
:1059F00000290ED18168294381600120FFF7D6FF7D
:105A000000F086FF07460CE000F082FFC01B0A286A
:105A100007D9606D30436065A06D2843A065012003
:105A2000F8BD20680068C043C007EDD10020F8BD74
:105A30001700008010B500231A4603E0845CE318C9
:105A40009BB2521C8A42F9D3D84380B210BD0000E9
:105A500010B5034800F01CFD024800F019FD10BD10
:105A6000C01500207815002030B5446C1C252C4052
:105A70000125A540046C6560046863608368102B91
:105A8000036803D099600068C26030BD9A60006806
:105A9000C16030BD1449012048720A4602205E32BE
:105AA000507203203C3A507204200E3A50720F4854
:105AB0000D4B0078087022310870203108770C49AE
:105AC0005A1C0878587149789971233318715971A3
:105AD000203318775977107551751A461E32107594
:105AE000517510765176704750110020D700002074
:105AF000F400002010B503F0B3F9202003F05CFAA5
:105B0000012004F09DFA002003F056FA044804F046
:105B10003BF9044804F0EAFB002004F01FFC10BD30
:105B2000C00000208380000070B50520012100071F
:105B300000F0DEFE0025154C002800D06560144EF4
:105B40000221304600F0D4FE002817D10120207039
:105B50007F20C005A0600F48808F002805D001215C
:105B600000228902304600F0CCFE0B4865600088B8
:105B70000A2148430949088003F004FE012000F08F
:105B8000EFFD022000F0ECFD70BD00000C010020D4
:105B900000040050500D0020E4000020F000002020
:105BA0007047000010B5084900224A6107494B6858
:105BB0004C1523434B604B68082423434B60C009BA
:105BC000C001026010BD0000081600200020024045
:105BD0007FB500250C460646039500F091FDE009CF
:105BE000029003A901960095684600F021FD002867
:105BF00004D000F059FD002004B070BD00F054FD49
:105C00000120F9E710B5002302E0C45CCC545B1C12
:105C10009342FAD310BD000010B5214A00219069CB
:105C2000C305204804D541690223194341619115F8
:105C300093699B0505D543690124234343616302AE
:105C4000194393695B0505D54369082423434361E0
:105C5000E301194393691B0505D5436904242343D4
:105C600043616302194393699B0405D5436910247A
:105C7000234343616302194393699B0304D5446939
:105C800020231C43446119439369DB0305D5436911
:105C9000402423434361A0020143916110BD0000F1
:105CA000002002400816002070B5054600F030FEC6
:105CB0000646184C0AE0681C08D0002D04D000F0FD
:105CC00027FE801BA84201D9032070BDA069C00730
:105CD000F1D1A069800701D50220A061A069C005AB
:105CE00011D4A06980050ED4A06940050BD4A06929
:105CF000000508D4A069800405D4A069800302D4FB
:105D0000A069C00303D5FFF787FF012070BD002005
:105D100070BD000000200240F8B517460026054679
:105D20000C4600F0EDFC09E029460220226800F054
:105D3000C9FC002804D1241D2D1D361DBE42F3D3FD
:105D400000F0B2FCBE4201D20020F8BD0120F8BD37
:105D500010B5084902460020054B497905E044008A
:105D60001C5B944203D0401CC0B28842F7D310BDE4
:105D7000781200205800002010B500F0BEFD10BDC4
:105D800010B5094800F086FF80B2FFF777FC074A9C
:105D9000074BFFF76DFB0022064BFFF7D1FBFFF728
:105DA000B3FC80B210BD000070140020F853E3A5CE
:105DB0009B843E4000408F4070B5384C3648217F70
:105DC0000175617F417536490A78027649784176D6
:105DD00031490520133148720A2004F077FA7D20FA
:105DE000C00004F08DFA2C49002213310C2004F07D
:105DF00057FB00210C2004F065FB022004F0B6FAEA
:105E0000284D00210F2004F0E1F92842E062F8D08B
:105E1000E06A411C30D0400430D58122D2010021FB
:105E20000F2004F012FB0021102004F0CFF94106EE
:105E30001948490E0022633004F0FEF9164D63350F
:105E4000687A052817D102221549681DFFF7BAF9AB
:105E5000002810D11148AE7C66710422691C4030C4
:105E6000FFF78CF929461331084672005130FFF7CD
:105E700085F90320207070BD02F00AFA0A480188F3
:105E8000608B0546FFF734F908480088414308480D
:105E90006D1E0180658370BDB11100205800002087
:105EA000F400002000D02724E0000020DE000020C5
:105EB000DC00002010B5084800F096FA0A210648D8
:105EC00000F032FA044800F01DF9800503D50248BD
:105ED00000F01AF980B210BD14140020F8B52F4D4F
:105EE00000220121284600F00CFDFFF7E3FFFFF739
:105EF000AAFB2B4E3146FFF7CBF92A4C0122A060BA
:105F00001146284600F0FDFC2749A068002588427C
:105F10003EDB2078254F002815D02570FFF7CAFFFB
:105F2000FFF791FB3146FFF7B3F9A060FFF70AFCDA
:105F300000223B46FFF78EFA00221D4BFFF798FA2E
:105F4000FFF714FC6060A068FFF7FCFB00223B46F3
:105F5000FFF780FA174A184BFFF78AFA06460F46F2
:105F60006068FFF7EFFB134A144B5242FFF780FAC9
:105F700032463B46FFF7CAF9FFF7F8FB104960606D
:105F8000884201DD616004E0FF21C905C84200D3F9
:105F900065606068FFF780FBC0B2F8BD0004005088
:105FA00000401B44300000200000604000000C4016
:105FB00000E064403333333333B33040CCCCEC3F78
:105FC0000000C842F8B5054604464035287C002646
:105FD000012808D001202874206881688907890F6A
:105FE00001290ED101E00220F8BD0168C90708D0DF
:105FF000606D20210843606501260020287430462A
:10600000F8BD616DFF2201329143022211436165A7
:10601000C1688907890F0091C16889088900C1603A
:106020002068816892071143816000F071FC074687
:106030000EE000F06DFCC01B0A2809D9606D02213A
:106040008843102108436065002028740120F8BDB2
:10605000206880680028ECDB2068C168009A114342
:10606000C160606D80088000401C6065C5E700006D
:10607000F8B506460D464036317C01290DD0012188
:10608000317401688A68520709D5416D2022114395
:106090004165002030740120F8BD0220F8BD174B87
:1060A0006A68D80547109A42154C8A6A2B6812D044
:1060B0005B035B0B1A438A622968490305D5A16813
:1060C0000143A1600A20FFF771FC2868800312D504
:1060D000A06838430EE05B035B0B9A438A62296831
:1060E000490302D5A1688143A1602868800302D5D5
:1060F000A068B843A06000203074F8BD0110000013
:1061000000270140406D70470068006C7047000038
:1061100070B5040006D0606D264600254036002884
:1061200002D006E0012070BDA5653574204600F060
:10613000D3F8606DC00603D421688868400705D590
:10614000606D1021084360653574EBE7606DFF22D8
:106150000132904302221043606588688207920FE3
:106160005B48012A02D10A68D2072BD10323626857
:106170009B079A4205D05B429A4202D05B009A424A
:1061800009D10A69920092080A6121680A69636864
:106190001A430A610CE00A69920092080A61816858
:1061A0000F2292049143816081686268114381608B
:1061B0002168CA6818239A43CA602168CA68A3681C
:1061C0001A43CA6081680122520691438160816846
:1061D000A28E52061143816020688168C90004D4F0
:1061E000816801221207114381602068C168394A21
:1061F0001140C1602069E168022825D000200143D8
:10620000204620300278037B52035B001A4311437F
:10621000226B1143A26992031143E269D203114335
:106220002268D3681943D160616A0A46FF3AC23ACC
:1062300005D0A26A11432268D3681943D16042781D
:106240000121012A02D00BE00420D8E700780028C1
:1062500023D0606D202210436065A06D0843A065C7
:10626000E06B012820681FD00169C90703D00169CC
:1062700049084900016120684169C908C9004161B4
:1062800020684169A26B11434161A565606D80087A
:106290008000401C6065002070BD2068C26801233A
:1062A0001B041A43C260DBE70269FF239B009A4389
:1062B000026120680269236CA66C1A43636C334345
:1062C0001A430261206802690A430261D3E70000B1
:1062D000002701401902FEFF10B586B004461421C4
:1062E0006846FEF764FF0E492068884216D10D48C3
:1062F000416B421511434163C16A01221143C162DE
:10630000C06A694610400590022000900320019069
:10631000002002900520000700F02EFA06B010BD04
:106320000024014000100240F8B5044640692546AB
:1063300040350E4608280BD02068C068C00709D039
:10634000606D202108436065002028740120F8BD9D
:10635000082700E00C2700F0DBFA009011E0701C29
:106360000FD0002E05D000F0D3FA0099401AB042A9
:1063700007D9606D0421084360650020287403205C
:10638000F8BD206800683842E9D0606D01214902FB
:10639000084360652068C16809058A0F0C21002A3E
:1063A0001BD12022125D002A17D10268120714D5D2
:1063B000826853070122002B08DB43688B4343604C
:1063C000606D130298431043606506E0606D202302
:1063D00018436065A06D1043A065A069002801D135
:1063E000206801600020F8BD70B5044621680020D7
:1063F0008968490721D425464035297C01291CD0CC
:1064000001212974E169012904D02046FFF7E0FA4F
:10641000002811D1616D0A4A1140FF220132114357
:1064200061650021A165297422681C211160216821
:106430008A6804231A438A6070BD022070BD000080
:10644000FEF1FFFF70B50024014620314A79022A8F
:1064500003D00421C163012418E0026813680E25EB
:10646000AB431360026813685B085B001360436C06
:106470001C221340012215469D40036C5D604A7149
:1064800000220A71816B002900D08847204670BD28
:10649000F0B4016C0D6801680C68466C1C23042282
:1064A0001E401746B7402F420ED067070CD50C6828
:1064B000A40602D40C6894430C60416C19408A40D5
:1064C000016C4A60016B1AE00227B74002462F4078
:1064D0002032002F17D0A70715D50C68A40605D4C5
:1064E0000C680A25AC430C6001215171446C0221F7
:1064F0001C40036CA140596000211171C16A002940
:1065000018D0F0BC08470827B7402F4212D0240704
:1065100010D50C680E25AC430C60446C01211C4066
:106520000B46A340046C6360C1635171002111717B
:10653000416BE4E7F0BC704770B504003CD01F48E5
:10654000256814212818FEF7D3FD800060641C48DC
:1065500020640221204620300246417129681948F2
:10656000E3680140A0686669184323693343184310
:10657000A3691843E3691843236A18430843286052
:106580000121A0688903884210D00D488030836AB9
:10659000656C1C210D400F26AE40B3438362656CD1
:1065A00063680D40816AAB400B4383620020E06367
:1065B00001215171107170BD012070BDF8FFFDBF48
:1065C000000002400F80FFFFF8B504468C462030E3
:1065D00001790025012909D001260671417900279A
:1065E000012905D0077102252846F8BD0220F8BD13
:1065F00002214171E7632068016849084900016090
:1066000061462046FFF730FA206B002820680168B9
:1066100001D00E2205E00422914301602068016848
:106620000A22114301602068016831430160DBE701
:10663000F8B51A4E0546307C0F46012807D00120D8
:1066400030741748FFF730FB010002D021E0022030
:10665000F8BD0020C04338606C6814E02046FFF7A6
:10666000A1FA0F48FFF720FB01460E4842680823B5
:106670009A434260426843159A434260002901D020
:106680003C6006E08034A8686A68C0018018A042B7
:10669000E4D8002030740846F8BD00000816002039
:1066A00050C3000000200240054841680222114307
:1066B00041604168012211434160002070470000A1
:1066C00000200240F8B50C4C1646207C0F460128ED
:1066D00008D0012020740948FFF7E6FA00250028B9
:1066E00002D006E00220F8BD65613E600348FFF776
:1066F000DBFA2574F8BD00000816002050C3000026
:1067000011484168C9070BD0EFF3108172B60F4AE8
:10671000C2600F4AC26081F310884168C9070ED178
:10672000416889070DD5EFF3108172B6094A0261FD
:10673000094A026181F310884068800701D5012071
:10674000704700207047000000200240EFCDAB8969
:1067500005040302BFAE9D8C16151413704700008C
:1067600010B504494A69024202D04861FFF7F6FFBA
:1067700010BD000000040140F8B500230124A2E090
:1067800027469F403A4070D04D68022D01D0122D0F
:1067900014D1DD08AD002D1800952D6A5E07AC46BA
:1067A000F50E0F26AE46AE406546B543AC460E69C3
:1067B0007546AE4065462E43009D2E624D68012D04
:1067C00005D0022D03D0112D01D0122D16D18568D0
:1067D0000326AC465D00AE46AE406546B543AC46CA
:1067E000CE687546AE4065462E43866046680D7994
:1067F000BE43ED06ED0F9D403543456006685F00E2
:106800000325BD40AE46AE430D79B446AE07B60F84
:10681000BE4065462E430660C6687546AE438D6829
:10682000BD403543C5604D68ED004BD5294D6E6BBD
:1068300026436E639E08284DB6007519AC46AD68B8
:106840009E07360F0F27B740BD4305273F07B842C5
:1068500001D1002715E0214FB84201D1012710E0F6
:106860001F4FB84202D102270BE02BE01D4FB84268
:1068700001D1032705E01C4FB84201D1052700E0F4
:106880000627B7402F436546AF60184D2E684F6806
:106890009643FF0300D516432E606E684F689643FB
:1068A000BF0300D516436E60AE684F689643FF0283
:1068B00000D51643AE60EE684F689643BF0200D520
:1068C0001643EE605B1C0A681546DD4000D057E7B2
:1068D000F8BD00000010024000000140000400501C
:1068E00000080050000C0050001C00500004014043
:1068F0000069084000D00120704742694A40426167
:106900007047002A01D081617047816270470000A2
:106910000148006870470000180100200248016823
:10692000491C0160704700001801002010B508489C
:1069300000240168402211430160204600F00AF85B
:10694000002801D0012401E000F0D0F9204610BD5C
:106950000020024070B5054609487D210024C90089
:106960000068FEF7C5FB00F065FE002801D0012499
:1069700004E000222946501E00F0D8F9204670BDE0
:106980001C01002070477047F8B5394C0126A078EB
:10699000401CA0702671E08A401CE08235480088C7
:1069A00002F0C4FA344DE888FEF74DFE3349FEF795
:1069B0006FFC334F3968FEF712FC38603148F1053F
:1069C000006800270090884210DB208AFEF73BFE1B
:1069D00001467F20C005FEF75BFC0099FEF754FCE2
:1069E0002849086028480221017001E02648077004
:1069F00002212648FFF77CFF002809D027632048A2
:106A0000234A016823480091914212DD067011E08B
:106A1000E888FEF718FE1949FEF73AFC216BFEF7ED
:106A2000DEFB1D4920638842E9DB1D491B48C86025
:106A3000E5E70770688F401EFEF7FAFD0099FEF744
:106A4000B1FE05D86079002802D01648067001E032
:106A500014480770688FFEF7F6FD09490968FEF7CC
:106A6000A1FE04D26079002801D003F01BFEF8BD1E
:106A7000D400002072000020500D002000007A4455
:106A800010010020140100206900002000040050C3
:106A90000000F0425E0000200000A0400400FA0563
:106AA00000ED00E06B000020704770B505000DD0D0
:106AB00002202C462034A073284601F00BFA284609
:106AC00000F0BEF80020A073607370BD012070BD9F
:106AD0007047704710B5044600680168C943C9078C
:106AE00008D18168C943C90704D10121416020460A
:106AF000FFF74AFF20680168C943890708D4816805
:106B0000C943890704D4022141602046FFF73AFFB8
:106B100020680168C943490708D48168C943490707
:106B200004D404214160204600F0DEF820680168AA
:106B3000C943090708D48168C943090704D4082157
:106B400041602046FFF7B0FF20680168C943C906CD
:106B500008D48168C943C90604D410214160204685
:106B6000FFF711FF20680168C943890608D48168CE
:106B7000C943890604D4202141602046FFF7A9FFBC
:106B800020680168C943490608D48168C943490699
:106B900004D4402141602046FFF79AFF10BD000059
:106BA000F8B5040005D025462035A87B002802D082
:106BB00006E00120F8BD00206873204600F052F87E
:106BC0000220A8732068C26884466368012B04D041
:106BD0000120A16AC005814201D11E2082431548CF
:106BE0006169814201D0144802401448A6680240FD
:106BF00018463043676A266A3E433043A66A3043EC
:106C00001043012B03D00122D205964203D1236900
:106C1000E2681A431043074A914205D0A269114322
:106C2000E2690243084610436146C8600120A87328
:106C30000020F8BDFFFF00003F1FFFFFF8F119FF24
:106C400010B500680549884207D10548816B4900A5
:106C5000490881630D2000F055F810BD007C00400C
:106C60000010024010B50068084988420CD108485D
:106C7000816BC20411438163002201210D2000F0C9
:106C800055F80D2000F048F810BD0000007C0040D1
:106C9000001002400068C0697047000070B502240F
:106CA000034620339C730F4C2568E604354325606A
:106CB0000468E568B6123543E5600568AE680124EE
:106CC0002643AE6005682E6926432E610568A961DA
:106CD00001684A61006801690422114301619C73E3
:106CE000002070BD00040140704700000448416B63
:106CF000012211434163816B020411438163704798
:106D000000100240C106C90E0120884001490860F8
:106D10007047000080E100E0C106C90E01208840F4
:106D2000014908607047000000E100E010B501F083
:106D30008DFA10BD02494A6882434A6070470000DC
:106D400000700040024801688215114301607047DD
:106D50000070004002494A6802434A6070470000E0
:106D60000070004005480168022211430160044898
:106D7000016904221143016130BF70470070004077
:106D800000ED00E00A4B1A689208920002431A6074
:106D900008480369042213430361012906D040BF58
:106DA00020BF20BF016991430161704730BFF9E7FF
:106DB0000070004000ED00E0F8B504460078544D46
:106DC000800672D5524E0027403EB06BC00004D4FE
:106DD000B06BA9050843B06301274E480168C90597
:106DE00011D40168821511430160FFF791FD0090F5
:106DF00005E0FFF78DFD0099401A642837D8454813
:106E00000068C005F5D532680321090560680A40AD
:106E10000140914208D08103890F032904D13168D0
:106E2000890301D50120F8BD2A69032109040A401C
:106E300022D0084090421FD0207880061CD52869B7
:106E40002A6988430121C9040A432A612A698A43BD
:106E50002A612861C0050FD5FFF75AFD009008E0B0
:106E6000FFF756FD0099411A2B48814201D90320B2
:106E7000F8BD28698005F3D561688803800F032871
:106E800005D132680005824301400A433260286917
:106E9000032261681204114008432861002F04D0C6
:106EA000B16B012000078143B1632078C00705D092
:106EB000E868A168800880000843E86020788007BF
:106EC00005D5E8680C218843E1680843E86020782C
:106ED000400706D5E86803218902884321690843F1
:106EE000E8602078000706D5E86803210903884395
:106EF00061690843E8602078000606D5E868032148
:106F000089048843A1690843E8600020F8BD0000B7
:106F1000401002400070004088130000F8B50E4693
:106F200005007DD053480068C007C00FB0420AD2A8
:106F30005048016849084900314301600068C007B2
:106F4000C00FB04271D128784B4C800705D5E0685E
:106F5000F0218843A9680843E0602878C00752D030
:106F60006868022817D0032818D02168012818D093
:106F70008905002959DAE168890889000143E1603F
:106F8000FFF7C6FC69680746022912D003291CD006
:106F9000012926D033E021688903EAE721688901C5
:106FA000E7E74907E5E7FFF7B3FCC11B3348814238
:106FB00023D8E0680007800F0228F4D123E0FFF710
:106FC000A7FCC11B2D48814217D8E0680007800F3D
:106FD0000328F4D117E0FFF79BFCC11B274881422F
:106FE0000BD8E0680007800F0128F4D10BE0FFF711
:106FF0008FFCC11B2148814201D90320F8BDE06804
:107000000007800FF3D11B480168C907C90FB142BF
:107010000DD901684908490031430160006800E06A
:1070200003E0C007C00FB04201D00120F8BD2878AE
:10703000400706D5E068072109028843E96808434C
:10704000E0602878000707D5E0680721C902884377
:107050002969C9000843E06000F036F8E168084A91
:107060000906090F515CC840064908600020FFF777
:1070700071FCF8BD0020024000100240881300009F
:10708000DAA800081C010020044805490068C96806
:10709000044A4905490F515CC84070471C01002053
:1070A00000100240F3A80008044805490068C968B8
:1070B000044A8904490F515CC84070471C010020F4
:1070C00000100240F3A8000810B5184AD1680C203F
:1070D000084004280BD0082810D00C2810D0506885
:1070E0000004410F0120C003491C884010BD1068F6
:1070F000C00601D50E4810BD0E4810BD0E4810BD8B
:1071000088020E4B000F185C0902D368890F491CD6
:10711000DB0301D5084A05E01268D20601D5044A0E
:1071200000E0044A5043FDF7E3FF10BD00100240A9
:1071300000093D000024F40000127A00EAA80008CB
:10714000FEB505007ED0FE4CE7680C20E6680740DF
:107150000120000406402878C00747D0082F05D03A
:107160000C2F0AD101200004864206D1206880033A
:107170003CD568680028E5D038E001206968000443
:10718000814203D121680143216011E005230122DE
:107190001B0492049942216802D111432160F1E756
:1071A0008143216021680140009120689043206064
:1071B000686800280DD0FFF7ABFB009005E0FFF7F3
:1071C000A7FB0099401A64287AD820688003F6D576
:1071D0000CE0FFF79DFB009005E0FFF799FB00999D
:1071E000401A6428F0D820688003F6D428788007F5
:1071F00055D50923E868042F0DD00C2F01D1002E9E
:1072000009D000283BD02168994301432160FFF752
:107210007FFB064627E02168490701D5002891D069
:1072200061681F22120291432A69120211436160B0
:107230002168994301432160FFF746FFE168090691
:107240000A0F00E079E1BF49895CC840BE49086087
:107250000020FFF77FFB002872D120E0FFF758FBEA
:10726000801B0228B0D820684007F7D560681F212E
:107270000902884329690902084360600FE0206819
:10728000400840002060FFF743FB064604E0FFF79C
:107290003FFB801B022897D820684007F7D4287846
:1072A000C0065FD5002F0CD0A869002849D02068FF
:1072B000FF21013108432060FFF72AFB06462DE03D
:1072C000C0E02068800502D5A8690028A7D06068C2
:1072D000072149038843296A084360606068297F61
:1072E0000002000A090608436060286A410B012079
:1072F000C003491C8840E16809060A0F9149895C6E
:10730000C840914908600020FFF724FB002817D1EE
:1073100028E0FFF7FDFA801B0228A3D8206880052B
:10732000F7D56068072149038843296A08436060EC
:107330006068297F0002000A09060843606011E0C6
:10734000E1E02168FF20013081432160FFF7E0FA8E
:10735000064604E0FFF7DCFA801B022872D820689A
:107360008005F7D42878794E000724D5686900286D
:10737000306910D0012108433061FFF7C9FA00904D
:1073800005E0FFF7C5FA0099401A02285AD830697B
:107390008007F6D50FE0400840003061FFF7B8FAEB
:1073A000009005E0FFF7B4FA0099401A022849D886
:1073B00030698007F6D42878400765D50020029010
:1073C000A06BC00006D4A06B012109070843A0638D
:1073D000012002905E480168C90511D40168821538
:1073E00011430160FFF794FA009005E0FFF790FA6F
:1073F0000099401A642825D855480068C005F5D57D
:10740000FF20AA680130824203D131690143316112
:1074100011E001218902002A07D005231B029A42AC
:1074200003D132690A433261EFE732698243326144
:10743000306988433061A86800280FD0FFF768FAE8
:10744000009007E05EE0FFF763FA0099411A4148B7
:10745000814257D830698005F5D50DE0FFF758FA1D
:10746000009006E0FFF754FA0099411A394881422A
:1074700048D830698005F5D40298002804D0A06B64
:10748000012109078843A063686A002864D00C2F93
:107490003ED0012636060228206805D0B043206081
:1074A000FFF736FA05462FE0B0432060FFF730FAC9
:1074B000074604E0FFF72CFAC01B022822D82068F8
:1074C0008001F7D4E96AA86AE2680843296BFD23C2
:1074D0001B049A4311430843E06020683043206056
:1074E000FFF716FA054604E0FFF712FA401B0228E0
:1074F00008D820688001F7D52EE0FFF709FA401B75
:10750000022801D90320FEBD20688001F5D423E0C4
:107510000128F8D0E06801210904AA6A01409142DB
:107520000BD10F218904EA6A0140914205D1032160
:1075300089050840296B88420ED00120FEBD00005D
:1075400000100240DAA800081C0100204010024090
:1075500000700040881300000020EFE770B50400C1
:1075600007D0002625464035A662687C002802D058
:1075700005E0012070BD2E74204600F02FF8022097
:10758000687420680168402291430160A1686068C6
:1075900022690843E16811430843616901220843F5
:1075A000A169520211400843E1690843216A084376
:1075B000A16A084321680860A0690421000C084002
:1075C000616A0843216848602068C169920091435C
:1075D000C161666501206874002070BD10B586B079
:1075E000044614216846FDF7E2FD104920688842F0
:1075F00019D10F48416B821411434163C16A0122C2
:107600001143C162C06A002110400590E020009043
:107610000220019003200390029104910520694605
:107620000007FFF7A9F806B010BD000000300140C8
:1076300000100240094910B5401E884201D90120BE
:1076400010BD074C60610321081F00F0FFFD002002
:10765000A06107202061002010BD0000FFFFFF0097
:1076600000E000E070477047F8B502680446D06952
:107670001168936805072D0F5BD0DD07ED0FFF261E
:1076800021360E402E4367D0C60706D0CE0504D55E
:1076900001261662E26F3243E26787070222042660
:1076A000002F06DADF0704D027683A62E76F374316
:1076B000E767470706D5DB0704D023681E62E36F40
:1076C0001343E367020709D520220A402A4305D065
:1076D000236808221A62E36F1343E367E26F002A0C
:1076E0002FD0800606D5880604D5216E002901D04A
:1076F00020468847E06F21688968490601D4000761
:1077000024D5204601F09CFE20688168490619D5E1
:107710008168402291438160E06E002812D02049A8
:107720008163E06EFEF78EFE00280AD0E06E816B6A
:1077300006E0850610D58D060ED5216E1CE020468C
:107740008847F8BD2046FFF78EFFF8BD2046FFF7BB
:107750008AFF0020E067F8BDC50208D55B0206D5A8
:107760000120000510622046FFF77CFFF8BD0306EC
:1077700005D50B0603D5616E0029E0D1F8BD4006A2
:10778000FCD54806FAD51368204640218B43136088
:10779000202161670021616600F069F9F8BD0000F1
:1077A0009D93000810B5040003D0606F002802D03C
:1077B00007E0012010BD002170200155204600F097
:1077C00027F82420606720680168490849000160A3
:1077D000204601F07FFE0128ECD0606A002802D02C
:1077E000204601F0BDFC206841680922D202914385
:1077F0004160206881682A22914381602068016885
:10780000012211430160204601F010FD10BD00006F
:10781000F0B587B0064614216846FDF7C8FC2C4930
:107820003068884251D12B48416B012292031143A9
:107830004163C16A01221143C162C06A0025104040
:1078400005900320400200900220032701A9A1C156
:1078500004200490052069460007FEF78DFF1F4CA9
:107860001D48A560E56081C48027E560A7602020F1
:10787000256160610002A0611848083CFEF75CFECB
:10788000002801D0FEF78CF9F466A662144C124869
:107890002146143820600320606010200831A1C107
:1078A0006561A561E56120462562FEF745FE002879
:1078B00001D0FEF775F9B466002201211B20A662F3
:1078C000FFF734FA1B20FFF727FA07B0F0BD0000DE
:1078D00000380140001002403000024078150020BE
:1078E000C0150020F8B50446806F20284DD100292E
:1078F0000BD0002A09D00123A0681B03984206D1AF
:107900002069002803D1C80701D00120F8BD254611
:107910006035287C012838D0012028745820616502
:1079200002530026E6672220A067E06E002819D0E7
:107930001749C162E16E17480863E16E1648486353
:10794000E06E13468663676D21683A462431E06E27
:10795000FEF73AFE002805D01020E0672E742020A4
:107960006067D2E72E7420680168FF22013211435C
:10797000016020688168012211438160206881686C
:107980004022114381600020F8BD0220F8BD0000B4
:10799000F993000837940008B193000870477047C6
:1079A000FFB50446406F83B017460D4620285CD1D2
:1079B000002D0AD0002F08D0A168C001814207D154
:1079C0002069002804D1E80702D0012007B0F0BDEB
:1079D000204660300290007C012846D002980121A8
:1079E00001740020E06721206067FEF791FF2646C2
:1079F00040360190378277820120A16800038142DE
:107A000002D12069002802D02F46002511E000276E
:107A10000FE000228021204601F070FE002815D1E1
:107A2000002F15D02168387888627F1C708A401E2C
:107A30007082708A019B002806980090E9D100228C
:107A40004021204601F05AFE002808D00320BDE75F
:107A500028882168C005C00D8862AD1CE6E720209B
:107A60006067029900200874B0E70220AEE7704713
:107A700001490248C160FDE70400FA0500ED00E09D
:107A800010B505242407002204212046FEF739FF03
:107A9000002208212046FEF734FF0A2002F02DF9CB
:107AA000012204212046FEF72CFF0A2002F025F9CE
:107AB000002204212046FEF724FF10BD10B5052446
:107AC0002407002204212046FEF71BFF0122082183
:107AD0002046FEF716FF0A2002F00FF901220421CA
:107AE0002046FEF70EFF0A2002F007F900220421CB
:107AF0002046FEF706FF10BDF8B500240526074610
:107B000025463607002204213046FEF7FAFE0A20F9
:107B100002F0F3F8012204213046FEF7F2FE60067F
:107B2000040E08213046FEF7E3FE002801D0641C55
:107B3000E4B2052002F0E1F86D1CEDB2082DE1D3AE
:107B4000002F03D0FFF79CFF2046F8BDFFF7B6FFDC
:107B5000FAE770B5052605463607002204213046AF
:107B6000FEF7CFFE0024E80901D0012200E0002248
:107B700008213046FEF7C5FE6806050E0A2002F011
:107B8000BCF8012204213046FEF7BBFE0A2002F0B9
:107B9000B4F8002204213046FEF7B3FE0A2002F0BA
:107BA000ACF8641CE4B2082CDDD370BD10B505241C
:107BB0002407012208212046FEF7A3FE012204210A
:107BC0002046FEF79EFE002208212046FEF799FE81
:107BD0000A2002F092F8002204212046FEF791FECE
:107BE00010BD10B505242407002204212046FEF70D
:107BF00088FE002208212046FEF783FE0A2002F0BC
:107C00007CF8012204212046FEF77BFE0122082198
:107C10002046FEF776FE0A2002F06FF810BD70B520
:107C200005252D070024012208212846FEF769FEBC
:107C3000062002F062F8012204212846FEF761FEC8
:107C4000062002F05AF807E0641CE4B2FA2C03D9CB
:107C5000FFF7C7FF012070BD08212846FEF748FE48
:107C60000028F1D1002204212846FEF74AFE002018
:107C700070BD0000F8B501F009FB01F043FB464878
:107C80000068C069FEF77CF84449454E898F002999
:107C900014D044490A7801218902002A0AD0012A15
:107CA00004D0022A04D0032A08D103E0212801D2FB
:107CB000002200E001223046FEF723FE0121C90226
:107CC0003046FEF715FE0127FF03374D002400283C
:107CD00025D036480460E879002803D10120E871F6
:107CE00001F050FD2878632806D90022082130468B
:107CF000FEF707FE012205E0012208213046FEF7CB
:107D000000FE0022052039460007FEF7FAFD234D4C
:107D1000274E4035A88C274F012803D01CE0EC717A
:107D20000022EAE724486946088072B68021234889
:107D3000FDF74EFF002804D0022269461F48FDF7D8
:107D4000EBFF62B61EA001F0BBFDAC8402F046FD65
:107D5000642001F0CBFFFE60688C012808D10F4839
:107D60006C84048002F03AFD642001F0BFFFFE60E5
:107D7000288C012806D12C8402F030FD642001F00B
:107D8000B5FFFE600548124A0188914202D1C088C1
:107D9000002800D1FE60F8BDF8140020500D00202E
:107DA0000004005069000020D400002010010020D1
:107DB0000400FA0500ED00E0AAAA0000384A000815
:107DC000BDF8C8EBC9FDBCB6C4A3CABD0D0A00000E
:107DD000AA55000008B53721202000F06EF80321D5
:107DE000212000F06AF84021222000F066F80821E6
:107DF000232000F062F8AA21302000F05EF80A4843
:107E0000008FC1B2322000F058F80221332000F078
:107E100054F85F21202000F050F8684600F006F882
:107E20000A2001F06AFF08BD500D002010B5014680
:107E30000F2000F021F8002800D0012010BD10B55F
:107E40000446FFF7B3FE3220FFF783FEFFF7E7FE9D
:107E5000E0B2FFF77EFEFFF7E2FEFFF7A7FE33205A
:107E6000FFF777FEFFF7DBFE0020FFF745FE044635
:107E7000FFF7B7FE204610BD10B50C46FFF7DFFF39
:107E80002070012010BD70B50D460446FFF78EFE30
:107E90003220FFF75EFEFFF7C2FEE0B2FFF759FEA9
:107EA000FFF7BDFE2846FFF754FEFFF7B8FEFFF7C9
:107EB00098FE0A2001F021FF70BD10B5FFF7E3FF27
:107EC000012010BD10B50248FEF704FE10BD0000F1
:107ED00070140020FEB50446002572B60068394AC9
:107EE000831804D13849CD68032189040D40816885
:107EF0000191C168009141698669002B08D132481F
:107F00004038836AC7043B438362836ABB4383620E
:107F10000846304348D02B482368C34205D12A483D
:107F2000C368032292049343C360002917D02068DA
:107F3000026901231A43026120684161FEF7E8FCEF
:107F40000746FEF7E5FC2168C01B0968090703D452
:107F50007D21C9008842F4D9216808204860002E9C
:107F600017D02068016901221143016120688661F0
:107F7000FEF7CEFC7D270646FF00FEF7C9FC216810
:107F8000801B0968C90601D4B842F6D921681020BF
:107F900048600C482168C14206D10B48C1680322E1
:107FA000920491432943C16020680169490849004E
:107FB000016121680198886021680098C86062B6F4
:107FC000FEBD00000084FFBF401002401CB5002130
:107FD00016480091144A01910260C1631205426083
:107FE000816007228263012202610246C160203261
:107FF0001170FF235170C2334362816211730163B8
:108000008161042241634261C161FEF781F8084841
:1080100000908013019069460448FEF729F800217A
:108020000248FDF7CFFF1CBD0024014014140020BE
:108030000200000408B50848016B012211430163E6
:10804000006B01211040009000220A20FEF76EFE16
:108050000A20FEF761FE08BD00100240F0B587B0AF
:1080600014216846FDF7A3F84C48C26A04210A436C
:10807000C262C26A0A400592C16A80273943C1625E
:10808000C16A39400591C16A01252943C162C16AAB
:1080900029400591C16A02263143C162C06A2A465D
:1080A0003040059005201C210007FEF72AFC012224
:1080B0003B493C48FEF725FC00223B493948FEF786
:1080C00020FC91210520002209020007FEF719FC7F
:1080D0003648019000240520694600950294000767
:1080E000FEF74AFB032001900520694600960294A2
:1080F0000007FEF741FB0C200090112001900320A7
:1081000003900520029469460007FEF735FB102016
:108110000090052069460396019502940007FEF73A
:108120002BFB1120019002946946009503941D4891
:10813000FEF722FB1E4801906946009602951948F9
:10814000FEF71AFB1B4800900294694601950394C0
:108150001448FEF711FBE8026A4651C2694611480D
:10816000FEF70AFB91200002009005200294694668
:10817000019503940007FEF7FFFA69460948009746
:1081800002950194FEF7F8FA002201210520FEF77E
:10819000CDFD0520FEF7C0FD07B0F0BD0010024088
:1081A000010600000004005008300000000011101B
:1081B000000021100836000010B50F4C0D4820605B
:1081C000FF20053060600020A060E06020616061F9
:1081D000E0610121206249026062A161A062072082
:1081E000E0622046FFF7BAF9206801684022114397
:1081F000016010BD00300140A014002000B585B022
:1082000014216846FCF7D3FF0E480D490160E121B7
:108210004902416000218160C160016181610C22DD
:10822000C161426101623021416201210903816320
:108230004900C163FFF7B6FA01F09EFA05B000BD30
:1082400000380140F8140020704700008307FF2227
:10825000DB0E9A408907090E994000280BDA0007C7
:10826000000F0838830808489B001818C369934317
:108270000B43C3617047830804489B001B181868B0
:10828000904308431860704700ED00E000E400E010
:10829000BFF34F8F04490348C860BFF34F8F00BF3F
:1082A000FDE700000400FA0500ED00E0F0B587B03E
:1082B0000A2002F00BF87D20C00002F021F8F94CF2
:1082C0000025A570607B0C2801D30B206073012270
:1082D000052051020007FEF714FB0026F248E67065
:1082E000F24D00782871F249A079097840000843DE
:1082F000E17C89000843E871A06AE870401CA06234
:1083000060792946A8744200B4310846A138FCF7C8
:1083100035FF06206872E74829460078A872A07EDB
:1083200028731339207F0875607F487560790022B3
:1083300040001331153002F0B3F86079002140009D
:10834000153002F0BFF8022002F010F8EE71E6736B
:10835000A67201252573E672D748FEF79BFC2084A0
:108360000746E6706079FDF789F9D44AD44BFDF7EA
:108370007FF801F057FC0022AB07FCF7C7FFFDF7C1
:10838000C3F90006C10CC81980B2E90360848842B1
:1083900001D3401A6084CB4860632079401C20716F
:1083A000C548FEF777FCE083C0480C3006464236ED
:1083B00040300390ABE1C048FEF76CFCE083C24F55
:1083C0000BE0BD48FEF766FC80B2E083618C88421A
:1083D00003D3BE4A8918884206D300210F2001F03A
:1083E000F5FE3842E062ECD0E06A411C21D0400446
:1083F0007ED58122D20100210F2002F026F87D20B7
:10840000C00001F07DFF002001F02FFF00211020AF
:1084100001F0DCFE4106A548490E274600225030F7
:10842000616401F009FFA1485030417A0729C1D1A8
:1084300001E0FFF72DFF0222A549401DFCF7C2FE17
:108440000028B7D102F08FF879653C46386502F014
:1084500077F8F965B865F8786A46401CF870934873
:108460004D30017911704079507010880090B98BAF
:10847000884273D19749308A08800398808A208384
:108480008D48FEF707FCE08301F0B2FDFF23A26DEB
:108490005B04E06D0021D21848410006170A07432B
:1084A00079084900080E0902216660667F48636DFD
:1084B0000A30226D02F02CF86079E36D81007B4870
:1084C000A26D0818163002F023F87848636E123057
:1084D000226E02F01DF87548082141726079002271
:1084E000800072491C3001F0DBFF6079800000E001
:1084F00000E100211C3001F0E5FF384601F0DFFE0D
:10850000012001F033FF207202217348FEF7F0F9D9
:10851000002824D000216648624A0170B189118682
:10852000F0895086614F226B50376263FB7C1A07DB
:10853000120F032A00D062741A090026A274267151
:10854000584BA5729986D886002A17D00222604916
:10855000781DFCF737FE002803D00FE076E00121FC
:10856000D9E75248E573C571606C50491638C2B2FC
:10857000663108462274D230FCF700FEE572208B8B
:108580005649FF30C33080B2208388420CD949421B
:10859000401820834F487D220188D200491C89B2AF
:1085A0000180914200D306804A48218B06887D20B5
:1085B000C00070434018A0630690494830210778F6
:1085C0004848A77300884843FDF73DF800900A200B
:1085D0007043FDF738F80099FCF75AFE7F21C90572
:1085E000FCF7FDFDFDF758F880B23D497F1E08807D
:1085F000B84200D1E572A6841420205EFDF72AF867
:1086000006460F46E08BFDF739F8374A374BFCF743
:108610002FFF049005910698FDF71CF8059B049A1E
:10862000FCF718FF32463B46FCF770FEFDF748F8B2
:10863000E063608B00F07AFC207A002870D1002182
:108640000F2001F0C3FD0006F9D569E0FDF780FBBE
:10865000274A032111541349B28987000A86244806
:10866000F2894A86603839180398008B08802049BF
:10867000206B3039C8510D48E36D38181630A26DA3
:1086800001F046FF1A486038C159206B81423EDD37
:1086900000293CD02146002839D000988883022048
:1086A000207034E058000020D4000020C4110020C5
:1086B0000C010020E400002070140020B81E85EB9F
:1086C00051B8CE3FA086010000D02724983A000080
:1086D000F40000200801002000040050E70300001F
:1086E000EA000020EE000020F853E3A59B843E4002
:1086F000F01200203A4600210F2001F0A6FE60791A
:10870000E178401C814202D0002001F0AEFDE18BF7
:10871000608C814200D24EE6184A80188142FAD815
:1087200001F066FC164A00210F2001F08EFE207930
:108730000A2800D92570E07B002805D011490B7864
:1087400048788A78022B0ED00D4A002180320F2003
:1087500001F07BFE01210520002249020007FEF7FF
:10876000D0F807B0F0BD084BC91C1818FCF706FD7F
:1087700002F034F8642001F0B9FA5AE6983A0000A1
:1087800000D02724FC120020500D0020704700006C
:10879000F0B58DB0B54801900020C0430A90002686
:1087A0000A2001F093FD7D20C00001F0A9FD00200A
:1087B000AF4C0546A070AF4FAF480B90AE480022BB
:1087C000C23885730146142001F06AFE002114208E
:1087D00001F078FE022001F0C9FD00210F2001F018
:1087E000F5FC3842E062F8D0E06A0146401C18D03F
:1087F00048047DD58122D20100210F2001F025FE01
:108800000021102001F0E2FC41069B48490E0022A5
:10881000801C01F011FD9848801C417A022902D089
:1088200004E1FFF735FD944802229449C01DFCF78E
:10883000C9FC0028F4D101F096FE6165206501F0C5
:108840007FFEE165A065002E22D10B988C49008A3D
:10885000088089480126801E808A20838948FEF787
:1088600019FAE083208B8849FF30C33080B220831F
:1088700088420DD949424018814920830888824A9C
:10888000401C80B20B320880904201D30020088047
:108890000B98694682890A80C089488076490422FB
:1088A000C91C0846A238FCF769FCFF22A16D5204DE
:1088B000E06D0023891858410006090A0143084663
:1088C000029101F0FCFC029948084000010E0002F0
:1088D000616620666848636D9638226D01F018FE67
:1088E0006548E36D9238A26D01F012FE624800E027
:1088F0009EE08E38636E226E01F00AFE5E49002211
:10890000A0393C2001F0CCFD00213C2001F0DAFD33
:10891000012001F02BFD2072A0780121401CA070E5
:108920000520C9030007FDF727FA55487D22008876
:10893000D200014602905043228B0A398018A0636E
:108940000C9052480078A073049008B2E08400288C
:1089500003DA7D21C9004018E0844D4830210088A9
:108960004843FCF770FE05902620205EFCF760FE71
:108970000599FCF78DFC7F21C905FCF730FCFCF75D
:108980008BFE424980B208800499491E884201D179
:108990000120E0720298A0841420205EFCF75AFEA9
:1089A00005910690E08BFCF769FE3A4A3A4BFCF7DA
:1089B0005FFD079104900C98FCF74CFE079B049A0E
:1089C000FCF748FD059B069AFCF7A0FCFCF778FE37
:1089D000E063608B00F0AAFA0099019881420DDAF9
:1089E00000290BD024490422C91C0AA8FCF7C6FBA5
:1089F000022020700520607200980190207A0028E3
:108A000005D100210F2001F0E1FB0006F9D58022FD
:108A100000210F2001F019FD00206D1CEDB26070E7
:108A2000032D00D2CAE6002E08D01AE00120F4E798
:108A30001A4A00210F2001F008FDF7E7608B401E65
:108A40000104090C1648618302D00288914201D9C1
:108A5000008860831349608B0988401E484312498F
:108A600008800A98A0830DB0F0BD00003F420F00BF
:108A70005800002000D0272412120020F40000200B
:108A80000801002070140020E7030000EA00002025
:108A9000EE000020F853E3A59B843E40009027247D
:108AA000E0000020DE000020DC000020F8B53149A5
:108AB0002F48086001F032FE304C2F486080E0887B
:108AC000002801D16420E080208F0A2801D90220EB
:108AD0002087E08E3C2801D93C20E086284980B2DE
:108AE0000870284DE08F6871A08FA871A07AE87097
:108AF000A68805212E626981E7883846FCF7F8FAD6
:108B0000A88101463046FCF7F3FA8800081886B2BF
:108B10007D20C0002E817043FCF7B0FD1A4A1B4B2C
:108B2000FCF70EFDFCF7F0FDE8817D206E823946F2
:108B3000C000FCF7DDFA28820146C820FCF7D8FA0D
:108B400068830120E882FDF71BF9A882EA891049B1
:108B50001048FEF7A3F810A0296A00F0B1FEE188E2
:108B600011A000F0ADFE218914A000F0A9FEF8BD0F
:108B7000B1970008500000200A020000500D0020AC
:108B800000000020D4000020F853E3A59B843E4061
:108B9000FF7F000070140020B1EAC7A949443A20C1
:108BA0002564202E0D0A0000CDA8D1B6BCE4B8F48F
:108BB0003A202564206D732E0D0A0000B5A5B4CEB1
:108BC000CDA8D1B6BBF9D5BECAFDC1BF3A20256438
:108BD000B8F62E0D0A000000F0B5904D85B00120CA
:108BE00028808F4FC8208F4C3880E079401CE0717E
:108BF000C00706D0608B411E6183022801D2C820C5
:108C00006083608B00F092F90A2001F05FFB7D2009
:108C1000C00001F075FB02218348FDF769FE0028C2
:108C200038D00020814980000978824E49000843ED
:108C30007F4909780843B072102070727E48C1885D
:108C40007D20C000FCF754FA70737C487A490078A4
:108C5000B07330460B308A780270C9784170411C7D
:108C600075482030027ECA70407E087172482230FA
:108C7000027E4A71407E887100220C39152001F075
:108C80000FFC0021152001F01DFC022001F06EFBFD
:108C90006B4E03E00120C5E7FEF7ECFF00210F203B
:108CA00001F094FA3042E062F6D0E06A411C7DD0D7
:108CB00040047CD58122D20100210F2001F0C5FBA8
:108CC0000021102001F082FA41065A48490E002284
:108CD0005030616401F0B0FA564E5036707A112867
:108CE00065D102225749701DFCF76CFA00285ED14D
:108CF000F01E027969460A7040794870B17A29807D
:108D0000C820FCF7F5F93880307B60834E4DB01EEB
:108D1000008A2880301F808A20834C48FDF7BAFFE4
:108D200080B2E0830390208B4949FF30C33080B28A
:108D3000208388420CD9494240182083288844491E
:108D4000401C80B20B312880884201D3002028804B
:108D50002D887D20C000218B68434018A0630290BD
:108D60003C48067828460A3800B2A673E0840028FA
:108D700003DA7D21C9004018E08438883021484357
:108D8000FCF761FC07462620205EFCF751FC3946C3
:108D9000FCF77EFA7F21C905FCF721FAFCF77CFC81
:108DA00081B22C48761E0180B14201E033E030E010
:108DB00001D10120E072A5841420205EFCF74AFC5A
:108DC000074601910398FCF759FC234A234BFCF713
:108DD0004FFB05460E460298FCF73CFC2A463346FC
:108DE000FCF738FB3A46019BFCF790FAFCF768FC6D
:108DF000E06368460088A0830E480E495030807CAE
:108E000060714200633108465130FCF7B7F9032026
:108E1000207005B0F0BDFFF73BFA0000E400002031
:108E2000EE0000205800002000040050D90000206F
:108E3000DA000020C4110020500D002000000020A6
:108E400000D02724F4000020080100207014002026
:108E5000E7030000EA000020F853E3A59B843E40AE
:108E600070B586B014216846FCF7A1F901250F4EB4
:108E7000ED03002229463046FDF743FD0120002482
:108E8000019002946946009503943046FDF774FC06
:108E90000320019002946946009503943046FDF743
:108EA0006BFC022000F022FF06B070BD00040050F1
:108EB00070470000F8B5044600206A461080194D3E
:108EC00055222A70AA226A700322AA70661DEE70CB
:108ED0002A716971144A49008918AC712246E81D4B
:108EE000FCF74CF9002007E029186A4689781288B7
:108EF00089186A461180401CB042F5DB611DA81C30
:108F0000FCF798FD01466846018029190078C87170
:108F100068464078087221460931024800F0A8FAF4
:108F2000F8BD0000B0130020500D002010B51B4C00
:108F3000E28A208A6178824201D3101AE082E28AB2
:108F4000608B134643435B182383132A02D150439B
:108F500040182083208B30214843642164304843EB
:108F60000F49E0620968401A0E494018A062FCF7F8
:108F700071FB0D4A0D4BFCF7E3FAFCF7A1FB0C4922
:108F80006062884202DD4A4280186062002801DA8D
:108F90004018606207490968486110BDD40000208C
:108FA00094000020F0D8FFFFF853E3A59B843E40D7
:108FB000FF7F000070140020034A1168382389B233
:108FC00099430143116070470030014010B5FDF72F
:108FD000A5FC10BD10B59AB034216846FCF7E7F83F
:108FE00014210DA8FCF7E3F81C2112A8FCF7DFF808
:108FF0001B4801680324E402A143C21489180160DC
:10900000FDF7A0FE17480169A14301610620009009
:10901000FF200130029001200390102004900220D4
:10902000099040040B90000100240C900A946846BB
:10903000FEF786F80F200D9003200E900F941094E9
:10904000012111940DA8FDF769FF812012900320E2
:1090500080041890149412A8FDF7AEFE1AB010BD4B
:109060000070004040100240104801688215114312
:109070000160C1680E4A1140C16001680D4A11408B
:1090800001608168490849008160016801229204F9
:1090900091430160C168FD2212049143C160002127
:1090A00001610649044888607047000000100240D2
:1090B0000C40FF88F6FFF6FE0050000800ED00E0CF
:1090C00070B501F097F8244C244DA06404E0FCF73F
:1090D00011FD01F08FF8A064A842F8D12078012694
:1090E0000525F6032D07002806D001280CD00228FC
:1090F00017D003282CD129E0012231462846FDF75C
:1091000000FCFFF769FD06E0012231462846FDF725
:10911000F8FBFFF73DFB002231462846FDF7F1FB47
:1091200016E0607A0122401E607231462846FDF743
:10913000E8FBFCF741FE002231462846FDF7E1FB43
:10914000607A002804D10120207001E0FFF7AEF81A
:1091500000F036FF70BD0000580000203001CADE6C
:1091600010B5818CC90707D001684A6801235B04E8
:109170009A43836A1A434A60818C890707D501683C
:109180004A6801231B049A43C36A1A434A60818CCC
:10919000490707D501684A6801239B049A43036B7A
:1091A0001A434A60818C090707D501684A68012380
:1091B000DB039A43436B1A434A60818CC90607D587
:1091C0000268916801231B039943836B19439160E3
:1091D000818C890607D501688A6801235B039A435D
:1091E000C36B1A438A60818C490612D503685A689A
:1091F00001210905046C8A4322435A60026C8A42A9
:1092000007D10268516803235B059943436C1943F6
:109210005160818C090607D501684A680123DB0487
:10922000806C9A4302434A6010BD0000F8B50026E6
:109230000446C667FDF76CFB054620680068124FC0
:10924000000709D501212B46002249052046009739
:1092500000F054FA00280DD12068006840070BD5B3
:1092600001212B46002289052046009700F046FA8E
:10927000002801D00320F8BD20206067A06760347B
:1092800026740020F8BD0000FFFFFF01F8B5184C60
:10929000C826E078002829D16079002826D101204D
:1092A0006071144D686B002700281ED0686BC821C0
:1092B000081A15E01048E168405C616988470F486A
:1092C0000A21008848430E490880E068401CE0609D
:1092D000E068C82800DBE760696BC820401A761E8A
:1092E000E168814201D0002EE4DC6771F8BD000026
:1092F0003C00002000000240880C0020E400002018
:10930000F000002070B5224CE07800283FD1207991
:1093100000283CD1012020711E4EF169002509066C
:10932000002933DA2156625791420AD1F06940068A
:109330002CD5A079002829D0A5712089401C208136
:1093400024E0A179002903D1A0710A2000F0D5FC06
:1093500000202056CC2148430F494218206912189A
:109360001279B262401C00222061A256CC235A43DB
:10937000895881420ADC25612078401C20702078C1
:109380000E2800D12570A078401CA070257170BDFA
:109390003C000020003801406001002010B5806AC8
:1093A0000022014640314A834A82FEF75CF910BD33
:1093B00070B5846A606FA56F216889680026090608
:1093C000002906DA212804D152200653204600F055
:1093D00047F820688068400606D5222D04D15A201F
:1093E0000653204600F02CF8E06F10210843E06798
:1093F0002046FEF738F970BD10B501460968806A4D
:109400000968890614D400225A210A5201680A68A0
:10941000FF2301339A430A6001688A6852085200A8
:109420008A6001688A6840239A438A6020218167A4
:10943000FEF7B4FA10BD10B5806AFEF7B0FA10BDA1
:1094400001680A68FF2321339A430A6001688A6829
:10945000520852008A60202181670021016670470E
:1094600001680A68C0239A430A6020214167704757
:1094700070B5164CE278002A0CD12279002A09D165
:109480000122E2700025C82903DC0222A256002A2C
:1094900001DCE57070BD0123E356CC2253430C4A36
:1094A000D1500123E356CC2673439B180A4601464C
:1094B000181DFBF763FE6078401C607060780E2812
:1094C00000D16570A078401EA070E2E73C0000204B
:1094D00060010020F8B504462669A268E7693243B6
:1094E0006669102000253E432368324378491E6890
:1094F000784F3E4016431E6023685A6803263603A1
:10950000B243E66832435A602368A2698B4201D0B5
:10951000266A32439E680B273F02BE4316439E6075
:109520006D4E23686D4AB3420CD1D2689207920FF8
:1095300006D0012A38D0022A34D0032A20D11EE0D6
:1095400001201DE0664EB3420AD1D2680C2632409B
:1095500026D0042A28D0082A24D00C2A10D10EE0C4
:109560008B420DD1D66803229202164018D00122F8
:109570009202B61A18D0B61A14D0964200D108201A
:10958000564A0126403A574FF6038B4236D10028FF
:109590000CD002280DD0042812D008281FD11CE0BE
:1095A0000020EDE70220EBE70420E9E7FDF76CFD82
:1095B00008E01068C00601D5384605E04A4803E0D7
:1095C000FDF782FD002873D0626851005118814276
:1095D00005D81103814202D303E03046F4E70125A8
:1095E00066E0010E06025008002330185941FBF7CF
:1095F00095FD03210902411A3C4A55E0E169B14257
:1096000032D1030000F083F909070A0D062506068A
:10961000062B0600E3E7FDF737FD1CE0FDF744FDF0
:1096200019E010686168C00602D54808304A01E0B8
:10963000304A48088018FBF75BFD80B201462E4A8D
:1096400010399142CBD8511C01400007400F08430C
:109650002CE0FDF739FD616840004A08EAE76168DF
:10966000012248081204E5E7030000F050F9090759
:109670000A0D06260606062C0600B0E7FDF704FDD7
:109680001DE0FDF711FD1AE010686168C00602D503
:109690004808C01902E014484A081018FBF728FDD2
:1096A00080B20146144A1039914298D82168C860A6
:1096B0000020206660662846F8BDFDF705FD61685C
:1096C0004A088018EAE7616848088019E6E7000060
:1096D00000480040F369FFEF0038014040100240AD
:1096E0000044004000093D000024F400FFFC0F008E
:1096F00000127A000048E801EFFF0000FFB581B0DA
:1097000017460E4604460A9D09E0681C07D0FDF77F
:10971000FFF80499401AA8420CD8002D0AD02068FE
:10972000C1693046884318D00020B842EDD00020EF
:1097300005B0F0BD20680168FF22A13291430160AD
:109740002068816849084900816020206067A0671F
:109750000020603420740320EAE70120E5E70000E0
:1097600010B504491020096808620248FDF77CFF23
:1097700010BD0000F814002001490D2088707047CA
:109780003C00002010B507480A22018A514381831A
:10979000FEF750FCFEF732FDC82203490348FEF7EE
:1097A000A1F810BDD4000020880C0020F81400207F
:1097B000F8B53E4C002321783D4A1D46082910D0BB
:1097C000072947D0062950D0052952D0042953D063
:1097D000032954D0002956D0012958D002295AD043
:1097E0005BE0A17800264A1F04E0314FBF5DFB1803
:1097F0009BB2761C9642F8DB667927799A19511844
:10980000E3786278C9188918C9194018C04300065E
:10981000000E1AD1012E14D0022E16D1254824494B
:10982000C018FBF7ABFC00F0D9FF642000F05EFA33
:10983000BFF34F8F21492048C860BFF34F8F00BF4F
:10984000FDE759081046FFF735FB2570E570A57058
:10985000A571F8BDA1795054491CC8B2A071A17876
:10986000491F8842F5D1082001E060700720207070
:10987000F8BDE0700620FAE760710520F7E7A070F8
:10988000E5700420F3E7552807D10120EFE7AA2867
:1098900003D10220EBE7032803D02570E570A57003
:1098A000F8BD032020702071F8BD0000CB0000201F
:1098B0004C130020500D00200400FA0500ED00E0DC
:1098C0000FB410B503A9044B044A029800F002F942
:1098D00010BC08BC04B0184729A5000820010020CE
:1098E0002021020C01D010211046020A01D010469E
:1098F0000839020901D01046091F820801D010461C
:10990000891E420801D0881E7047081A704730B47B
:109910007446641E2578641CAB4200D21D46635D0C
:109920005B00E31830BC184702E008C8121F08C1EA
:10993000002AFAD170477047002001E001C1121FD0
:10994000002AFBD1704708B50021684601706B46BC
:10995000012202212C2000F087FD022168460170BF
:109960006B4601222C2000F07FFD08BD38B504466F
:109970006D20694608706B46012207492E2000F0D1
:1099800073FD0649002C01D0054A00E0054A2E204F
:1099900000F050FD38BD0000060800000618000069
:1099A000070600000716000038B504466B46022281
:1099B0000021362000F024FCB3212300FFF7A7FF8D
:1099C0000E0F08153A3A3A3A1C273A3A2F34483AD9
:1099D00000216846017040784108490014E069465A
:1099E000087880088000401C04E0694608788008F8
:1099F0008000801C08701DE0684602780A404832EA
:109A000002704178802001436846417012E0684648
:109A100002780A40027040784106490EF4E7694630
:109A200048780221084303E069464878FD21084050
:109A3000694648706B4601220021362000F014FD73
:109A4000012200AB11463620013300F00DFD38BD78
:109A500069460878CF21084069462030CAE708B532
:109A6000032168464170012101706B4602220021EA
:109A7000362000F0F9FC0122D20306212D2000F04F
:109A8000D9FC012000F032F90120FFF78DFF08BD5D
:109A900008B5020A69464A7008706B460222042122
:109AA0002D2000F0E1FC0320694608706B4601227E
:109AB00006212D2000F0D8FC0020694608706B4676
:109AC000012206212D2000F0CFFC0A212D2000F0DC
:109AD0007DFB08BDFFB58DB00446002506E02528B6
:109AE0000AD0109A0F999047641C6D1C20780028AA
:109AF000F5D1284611B0F0BD00270121484A009752
:109B000000E00743641C23780846203B984010423D
:109B1000F7D120782E2817D1042007436078641CE1
:109B20002A280CD10E98641C02C800910E900BE0FC
:109B300000990A22514330394018641C0090207863
:109B4000014630390929F3D920780028D1D064287A
:109B500008D0692806D075281ED0109A0F99904712
:109B60006D1C5BE00A200E99019001C90E9100283E
:109B700002DA40422D2102E0390504D52B216A4644
:109B80001172012103E0F90704D02021F7E70BAEA1
:109B90000B910DE00021FAE70A200E99019001C90E
:109BA0000E91F7E70199FBF7A3FA3031761E317079
:109BB0000028F7D103A8801B20300190780701D539
:109BC000009801E0012000900199884201DD401ACF
:109BD00000E000200027009006E002A8109AC05D77
:109BE0000F9990476D1C7F1C0B988742F5DB04E0B2
:109BF000109A30200F9990476D1C0099481E0090D4
:109C00000029F5DC05E03078109A761C0F99904712
:109C10006D1C0199481E01900029F4DC641C65E765
:109C200009280100F8B54A002B4B520DD6182B4AD3
:109C30000C460546142E2BDA002E12DA284BFBF7C1
:109C400065FB00221346FBF78BFE40D2002C03DAA3
:109C50000124E40700253AE02046284337D0214C70
:109C600014E0214F0B46F7403B402B4331D01C4BB7
:109C7000FBF74CFB00221346FBF772FE27D2002CA9
:109C800003DD01200005F0400419BC4300251EE05F
:109C9000332E1EDC33460027143BFF43DF4038429F
:109CA00017D00F4BFBF7DCFB00221346FBF758FEE7
:109CB0000DD2002C0ADD142E0CD03420811B012083
:109CC00088404019A84200D2641C0546BD43214685
:109CD0002846F8BD641CF9E701FCFFFF9C7500886D
:109CE0003CE4377E0000F03FFFFF0F007D2110B500
:109CF000C900484300F001F810BD002140E000BF5A
:109D000000BF00BF00BF00BF00BF00BF00BF00BF5B
:109D100000BF00BF00BF00BF00BF00BF00BF00BF4B
:109D200000BF00BF00BF00BF00BF00BF00BF00BF3B
:109D300000BF00BF00BF00BF00BF00BF00BF00BF2B
:109D400000BF00BF00BF00BF00BF00BF00BF00BF1B
:109D500000BF00BF00BF00BF00BF00BF00BF00BF0B
:109D600000BF00BF00BF00BF00BF00BF00BF00BFFB
:109D700000BF00BF00BF00BF00BF00BF00BF491C45
:109D80008142BCD370470000FEB50446002001901C
:109D900000906079734940000E5A61782578491E19
:109DA0007148CFB20163042D77D0072D75D0002103
:109DB0000291217801736C49E37901229205896946
:109DC000002B6CD0914381616748217A4173217ADD
:109DD00082698907890B0A4382610021042000F00F
:109DE00034FB324661492E2000F024FB3846FFF751
:109DF000BDFD5F4E0522705D810040185D4943182E
:109E000007212B2000F030FB5B49029801220B1840
:109E10000B21282000F028FB705D584980000A586B
:109E20000C21282000F011FBE079554980004018F2
:109E3000A1794900425A0221272000F0FBFA51483B
:109E40007E00825B0421272000F0F4FAE0790028EC
:109E500029D0A07804282CD0282069460872202216
:109E60000621272000F0E6FA02AB01222621272056
:109E700000F0FAFA444938014018E1788900425864
:109E80000821272000F0E1FAA17A601C627A090219
:109E9000114313D016E000E001E0012188E71143EF
:109EA000F608816190E764220621272000F0C2FABB
:109EB000E0E71020694608720246D1E73349017293
:109EC000090A4172417A007A0A02024320212720BE
:109ED00000F0B0FA2E4F0C2123203A6800F0B5FABA
:109EE000F01982880421232000F0A4FAA079002828
:109EF0000BD0E0792749012243180021212000F0EE
:109F0000B3FA03200190012000902A07120F1001DC
:109F10000243607800218007000B0243019800058E
:109F200002430098400402432079C00640090243DE
:109F30006079C00602431F2000F087FAA07861789C
:109F40000123084302040848DB030261E179490365
:109F500019430A4302610021082000F076FA00202C
:109F6000FEBD0000A8A8000824010020042800006D
:109F700050A800080C0000202A00002058A8000863
:109F800078A8000884A8000888A8000841100000EC
:109F900070A800082C00002038B50C4607498A8BB1
:109FA000002102432C2000F045FA684604706B46FD
:109FB000012206212C2000F057FA38BD2401002090
:109FC00010B5FFF7C0FC10BD10B5044604213620C3
:109FD00000F0FCF80121C902002C01D0084300E088
:109FE000884302460421362000F02FFA10BD0000FD
:109FF00038B540206946087000210E2000F0E6F8D0
:10A000000446002211460E2000F01FFA6B46012282
:10A0100000210D2000F028FA074A00210F2000F04F
:10A0200014FA00F0EDF9224600210E2000F00DFA9E
:10A0300002480021017338BDF8FF272444010020A5
:10A04000FEB50546042069460870514C0020607535
:10A0500021462031206348710873A0836063A063A8
:10A0600000F0C8F84B4E206002E000F0C3F820601A
:10A07000B042FAD10020FFF797FC00F0BBF8464E43
:10A0800020603078242801D9243806E00621FBF727
:10A090002FF80622101A40010843020601040A4361
:10A0A00001020A430243B260706000211E2000F0EA
:10A0B000CCF900F09FF820606B460122002124209B
:10A0C00000F0D2F91E20FFF7E3FC86B2300AA0733D
:10A0D0000420FFF7DDFC074600F08CF8206038060E
:10A0E000000E0DD002206946087101AB0122122139
:10A0F0002D2000F0B9F9A08B012109030843A083AA
:10A1000000F078F820600620FFF7C2FC60600720AE
:10A11000FFF7BEFCA060F006C00E207501D1102034
:10A120002075C0B200F0DCF9E80707D0FFF797FC14
:10A13000A08B0121C9020843A0830AE00521362033
:10A1400000F02EF81549084002460521362000F09F
:10A1500071F90120FFF728FC0021042000F036F8F7
:10A16000A0610021262000F031F815218903084361
:10A1700002460021262000F068F900222621362020
:10A1800000F058F900F036F820600020FEBD000015
:10A19000240100203001CADE00000020FFFD000085
:10A1A00038B5094C89B280B26B46022200F028F81B
:10A1B000002806D1684640780102684600780818F1
:10A1C00084B2204638BD0000FFFF000038B50024EF
:10A1D000E44389B280B26B46042200F011F80028F3
:10A1E00006D103216846435C2202D418491EFAD5E1
:10A1F000204638BD10B500210846FFF7E7FF10BD27
:10A2000038B5002909D0402420436C462070C8B2DC
:10A210007F2906D8607002200AE069460870012094
:10A2200006E0802420436C466070C809A0700320BB
:10A23000694600F0ADFA38BD10B5144603460A462B
:10A2400021461120FFF7DCFF10BD10B503460522A3
:10A2500000211520FFF7D4FF10BD10B503460522DD
:10A2600000211720FFF7CCFF10BD38B505460020B0
:10A270006946087000F0C4F8FF2401342246002D1E
:10A2800001D00322120200210D2000F0D3F8002D8E
:10A2900013D06B46012203210F20FFF7B1FF684660
:10A2A0000078000709D5FFF7A3FE224600210D2004
:10A2B00000F0C0F80020C04338BD002038BD10B504
:10A2C000024601210A2000F0C0F810BD10B5044676
:10A2D00000211A20FFF77AFF000D22030005120B60
:10A2E000024300211A2000F0B0F810BD10B502465C
:10A2F00002492E2000F09EF810BD00000418000056
:10A30000F8B505466B46012203210420FFF778FFCC
:10A310000126114C3607002D0DD02A4600210C20B5
:10A3200000F088F8694608781021084369460870EB
:10A33000A069304307E069460878EF210840694684
:10A340000870A069B0430B46A061012203210420DC
:10A3500000F08AF8F8BD00002401002010B5024684
:10A360000021182000F066F810BD0000F8B507467F
:10A37000002568460570B807204C2E4600280ADAEA
:10A380008020694608706B46012200210D2000F0F4
:10A390006BF801202073F8076946087821D0062160
:10A3A0000843694608706B46012200210D2000F029
:10A3B0005BF803210F20FFF7F3FE8121C90008425B
:10A3C00019D04020694608706B46012200210D20FB
:10A3D00000F04AF80020FFF7F7FD00252673ED4353
:10A3E00009E002210843694608706B4601220021FA
:10A3F0000D2000F039F82846F8BD00004401002087
:10A400001CB56B46012203210F20FFF7F9FE6846B9
:10A4100000784022C1091040C9014000814208D0A3
:10A42000012069460871024601AB03210D2000F0AE
:10A430001BF81CBD08B56B461A70120A5A7089B217
:10A4400080B2022200F010F808BD38B500236C4637
:10A45000E254120A5B1C042BFADB89B280B2234659
:10A46000042200F001F838BD38B58024002909D055
:10A47000C02528436D462870C8B27F2907D8687068
:10A48000022009E0204369460870012004E02043CF
:10A490006870C809A8700320694600F0B5F938BD96
:10A4A00010B51446012312189B029A4202D90020CB
:10A4B000C04310BD0B46821E21460920FFF7D4FF82
:10A4C000002010BD10B5054A8905126901430A43F1
:10A4D00000210820FFF7B9FF002010BD2401002053
:10A4E00038B504466B4601220E212B20FFF788FE6B
:10A4F00068460078E10640094001C90E01436846FC
:10A5000001706B4601220E212B20FFF7ADFF38BDF5
:10A5100010B5002142541C06120A22431B0A491C92
:10A520000429F7DB10BD000013B501231A46694664
:10A530000248FDF735FA00981CBD0000F814002011
:10A540007CB5002425466846FFF77FFE0420694657
:10A55000220E2D02154322020C5C1443401EF7D537
:10A56000204629467CBD7CB5002425466846FFF779
:10A5700074FE04206946220E2D02154322020C5C53
:10A580001443401EF7D5204629467CBDFCF7CEF982
:10A59000FEF720FDFDF762FD3B493C48002522C047
:10A5A00005608561C5613A490562C1600838FCF7FC
:10A5B000F7FAFDF73FFDFDF721FEFDF7FDFDFDF785
:10A5C00005FD052601223607D1033046FCF799F92F
:10A5D000FEF76CFAFDF7FEFBFBF78CFAFBF75AFA75
:10A5E0000721B015FFF7D8FC2A4C0A21208A012246
:10A5F0004843A083170339463046FCF782F92348C5
:10A60000C82225498830FDF76DF9244E20790028AD
:10A6100036D0FEF7DFFC2571FBF760FC20700F28B9
:10A6200009D9012239463046FCF76BF9FEF748FD9F
:10A630000022394609E0012251033046FCF761F956
:10A64000FEF73EFD0022012149033046FCF759F98F
:10A65000FDF710FBA08B002801D0401EA0831048FE
:10A66000A18B00780843D1D10121C9023046FCF703
:10A670003FF90028CAD101210846FCF783FBC5E752
:10A68000FDF7F8FAC2E70000007C004070140020DB
:10A69000FFFF0000D4000020880C002000040050C0
:10A6A0004200002010B586B01748FCF7FEF91421CF
:10A6B0006846FAF77CFD15480090032001900020C1
:10A6C0000290052069460007FCF756F869461048D5
:10A6D000FCF752F869460F48FCF74EF8012108468E
:10A6E000FCF750FBFF2401342046FCF723FB0A490A
:10A6F00008680422104308602046FCF72BFBFCF797
:10A7000031FB06B010BD000070140020FFFF0000F8
:10A7100000040050000800500070004010B50122F5
:10A72000920218491848FBF76DFA16481749028833
:10A730008A4225D001807D21C90081804910C180D5
:10A740000A21018100211E224181D24382810122FE
:10A75000C2810184018241828182C182018381831D
:10A760001E23C38602230387782343878287C287F9
:10A7700002464032118451849184C18300F02EF846
:10A7800010BD0000500D002000FC0008AA5500007C
:10A79000F0B58C4600251026052109078E620E4C67
:10A7A00008E067467F5DE760A768FF07FCD0E768C1
:10A7B0001F706D1C8542F4DB0020074606E0E76051
:10A7C000A568ED07FCD0E5681D54401C9042F6D307
:10A7D0008E610020F0BD00000030014070B572B6FF
:10A7E0000124074DA40221462846FBF7F1F9002871
:10A7F00004D0224603492846FBF78EFA62B670BDA4
:10A8000000FC0008500D0020F0B50025102605279B
:10A810009C463F070B46BE620C4C06E0595DE1606A
:10A82000A168C907FCD0E1686D1C8542F6DB0020F9
:10A8300007E06146095CE160A168C907FCD0E168F6
:10A84000401C9042F5D3BE610020F0BD00300140B5
:10A850000000010203040005405C0000A05C04004D
:10A86000C06C0800805C0400E03F1E00E07D1E001C
:10A8700007A9022570889B880A00160001000600BF
:10A880000100020087008D002D001A3152001A339A
:10A890009A001A351D011A376B003B31BE003B335D
:10A8A0005E013B3596023B37000099599959EB51AF
:10A8B0008F421E45142E0080EB51F5283333E13AC8
:10A8C000703DE13AC235852BC2353333C235C235CE
:10A8D000AE47E13A5138A330513800000000000083
:10A8E00000000102030406070809030406080C100F
:10A8F0001820300000000001020304001CA9000819
:10A9000000000020240100002899000840AA000847
:10A9100024010020FC180000389900080000000005
:10A920000000000000000000070400091E080540A8
:10A930000826091040085608054008261D0400088E
:10A94000BE1D040008BED8BC401008000100000075
:10A950000000C842000000000000000000000000ED
:10A9600000000000000000000000000000000000E7
:10A9700000000000010000000000000000000000D6
:10A9800000000000000000005C1200000000000059
:10A9900000000000000000000000000000000000B7
:10A9A00000000000000000000000000000000000A7
:10A9B0000000000000000000000000000000000097
:10A9C0000000000000000000000000000000000087
:10A9D000000000000000000000000000020204006F
:10A9E00009090102008100000000000001000000D0
:10A9F0000006000000000000000000000000000051
:10AA00000000000000000000000000000000000046
:10AA10000000000000000000000000000000000036
:10AA20000000000000000000000000000000000026
:10AA300000000000000000000000200000000000F6
:04000005080050C1DE
:00000001FF
